:020000020000FC
:10000000F0C009C0189518957CC01895B0C0189517
:100010001895189518959F938F930F930FB70F937B
:1000200070FD14C091E080E98A179B0758F595E0B0
:1000300088E78A179B0730F171603327BB27AA270F
:100040000F910FBF0F918F919F91189590E08FE5C1
:100050008A179B07B8F490E08CED8A179B0790F005
:100060006030D9F06A95339533953E3019F47E7F30
:10007000EE24DD24BB27AA270F910FBF0F918F918C
:100080009F9118957E7F726067E0BB27AA270F912A
:100090000FBF0F918F919F9118951127552705E05C
:1000A00003BFE0E673FDEC0DE30F91918081A80F93
:1000B000B91F8894B795A795E0E673FDEC0DE30FA3
:1000C000B193A083DA0EEB1E339533953E3089F45D
:1000D0007E7F97E08EE98D199E09E0E673FDEC0DB9
:1000E000E30F9193808308E070277D7F7B7FEE2470
:1000F000DD24BB27AA270F910FBF0F918F919F91EE
:1001000018959F938F930F930FB70F931196219686
:10011000403011F401E008BB08E07027E0E673FD11
:10012000EC0DE40F9191808108E070278C179D07FA
:1001300030F00F910FBF0F918F919F9118954E3016
:1001400069F008B3000F08BB43954395DD27CC2722
:100150000F910FBF0F918F919F9118954427DD2725
:10016000CC270F910FBF0F918F919F9118959F935F
:100170008F930F930FB70F93183239F013950F9198
:100180000FBF0F918F919F9118957460E199FECFE9
:1001900000E0050F0EBBE09A9DB3E199FECF00E0B1
:1001A000050F03950EBBE09A8DB3E0E673FDEC0DF1
:1001B000E50F9193808308E07027E0E673FDEC0D76
:1001C000E50F9193808308E0702753955395503144
:1001D00011F4002703BF0F910FBF0F918F919F91D3
:1001E00018950FED0DBFF8940FEF07BB8C9A8D9A01
:1001F000929A939A00E40BBF02E005BF02E409BFA4
:10020000442733275527222711277727FF27BB2786
:10021000AA27DD27CC2704E1C02EE199FECF00E01C
:10022000020F0EBBE09A9DB3E199FECF00E0020FF2
:1002300003950EBBE09A8DB3E0E673FDEC0DE20F83
:100240009193808308E07027E0E673FDEC0DE20FE8
:100250009193808308E07027239523952031E9F658
:100260007E7F726067E0789400E00BBD04E60ABD13
:1002700009E00EBD05E003BF72FD02C0959801C004
:10028000959A71FD02C0949802C0949AF5CF839913
:10029000FF24F39489F7F894959A002708BB222746
:1002A00008E07027E0E673FDEC0DE20F919180818C
:1002B000E199FECF00E0020F0EBB9DBBE29AE19AEE
:1002C000E199FECF00E0020F03950EBB8DBBE29AD1
:1002D000E19A23952395203129F7959808E0702716
:0802E000839BFECF7894C8CF88
:00000001FF
